:1000000033222130840052280B1D0900A400030E66
:10001000A3008312051E0E28A5011328250FA50095
:100020004120FF30B000061C1728A6011C28260F0F
:10003000A6004120FF30B000861C2028A7012328FD
:10004000270FA70041202E082F0403192C28AF0FDB
:100050002C28AE0F2C28B1152B08031DAB032C0A3E
:10006000031935282C08031DAC03300803193B285D
:10007000B00B3B283116230E8300A40E240E0B1167
:100080000900FC30AE001830AF0008008207583479
:1000900000344C3400342034003420344D3448349F
:1000A0007A3400344330A0008001840AA00B542825
:1000B00007309F008316143085000330860004301B
:1000C00081008312FE20861CB11657228101A030C8
:1000D0008B004120B1118F30D5200230DB208B20E6
:1000E000B1196928311667228E30D5200030311DB4
:1000F0007C28331F7C280430DB203A301E223B2230
:1001000042302C22172244302C220A223A30252257
:10011000BC20992070288A30D5200630DB200800CA
:100120002C22922817225F30CD005030CE000A22B8
:100130000800B1104B09C039031DA528B114CB0923
:10014000CC090130CC070318CB0A3708CA000310CA
:10015000CB0D0310CC0D0318CB0A0310D3217B2148
:100160008130D520553084000930A0000008CB2014
:10017000840AA00BB628080038213A301E223530F8
:10018000252246302C22F321142135301E2208006E
:10019000CA20CA202030B500B6008615E4280130F8
:1001A000D5201830342208008130B500B600861101
:1001B000E42086150800B4004620FF390319080022
:1001C000CB203408013EDB288B13831603308600D6
:1001D00083120615F030B50506080C393504860083
:1001E00006110615B60EF030B60506080C393604B1
:1001F000860006114B3077218B17080086010F21EE
:100200000F210F2128308600061133222830D520F7
:100210000830D520CF200630D5200C30D528332209
:100220003830860006110800B210311550220F3008
:10023000CD00A030CE0017225D30CD00C030CE0002
:100240000A2248302C220122031935294830252260
:100250005C21C2304E214B084E214C084E21AE305D
:100260004E21FF304E2161213313B21831110800A5
:10027000331F3B294B215C21C3304E210830A000A5
:10028000762105147621050CB30D0510A00B40292D
:100290007221682161216E30AC000800B400083082
:1002A000A000B40D03187221031C6D216821A00B5E
:1002B00051297221682108000514722176216D21CF
:1002C0006A296D2176210514762172217621080094
:1002D00076210514762105100800851083168510F7
:1002E0008312080083168514831208000F30A100C2
:1002F000A10B7829080003101830A000D601D801FE
:10030000DB01DD01D30DD20DD10DDD0DDB0DD80DDF
:10031000D60DA00BAE295D0EDC005B0ED900580E89
:10032000D700560ED50031105530C3215630C321A9
:100330005730C3215830C3215930C32131145B30A9
:10034000C321A530DA005C30C3215D30C321B11C6C
:100350000800540884002D30800008005D30B7216B
:100360005B30B7215830B7215630B721822984003D
:1003700003300007B400B419800030300007B40027
:10038000B41B8000080084000F3000050319CC293D
:10039000303E8000311408003118C8292030800018
:1003A0000408D4000800D3014B08D1004C08D20047
:1003B0000830A000CA0C0318E229A00BDA29D101E9
:1003C000D20108000310ED29CA0C031CED294C08CA
:1003D000D2074B0803184B0FD107D10CD20CD30C0A
:1003E000A00BE42908004E08CC074D0803184D0F58
:1003F000CB0708004E08CC024D08031C4D0FCB0262
:1004000008004E084C02B4004D08031C4D0A4B0274
:10041000340408004D08CF004E08D0000130CE074C
:100420000318CD0A0122031C08004F301B2A0122A9
:10043000031808004D301E22B21408008400000882
:10044000CB00840A0008CC00080084004B08800020
:10045000840A4C088000080084000008CD00840A4B
:100460000008CE0008007630A100A201A20B362AB7
:10047000A10B362A0800CD010130861C1430CE00B5
:10048000A3222D18F321B4222D18FA210230861C44
:10049000C830CE009B222D18F321AC222D18FA2152
:1004A0004B09C039031D0800CB01CC01080083169D
:1004B0009B018312373084001130A0007E2280001F
:1004C00083169B0A8312840AA00B5E2A0800311E41
:1004D0000800311283169B018312373084001130DB
:1004E000A0007E2200020319772A000883228316C7
:1004F0009B0A8312840AA00B712A080083161C141D
:100500001A08831208008C1383169A001C158B138B
:1005100055309D00AA309D009C148B1783128C1FB0
:100520008F2A08001E30B4002A08AD002702BD2221
:100530002708AA00080064302502031CA32A4630BD
:10054000A5006630A42A3C30B4002808AD0025027E
:10055000BD222508A800080064302602031CB42A26
:100560004630A6006630B52A3C30B4002908AD00FC
:100570002602BD222608A90008000318C72A2D0854
:10058000053C0318C72A2D083402FF30031C030161
:10059000AD00080092222D1C08002B080319D12A57
:0805A00008001930AB00C72A66
:02400E00783FF9
:10420000FA004B0000004B0000004700E0005400A3
:104210006000000000004700E00054006000000063
:0242200000009C
:00000001FF
